:020000040000FA
:06000000FCEF13F01200FA
:060008001EEF13F01200D0
:060018001EEF13F01200C0
:06080000FCEF13F01200F2
:060808001EEF13F01200C8
:060818001EEF13F01200B8
:06082A000100402800005F
:08083000F500000002000000C9
:08083800D9CFE6FFE1CFD9FFA3
:10084000FD0EDBCF11F2FE0EDBCF12F2D950FD0F01
:10085000E96EFF0EDA20EA6EEE2A000EED22FD0EA2
:10086000DBCFE9FFDB2AFE0EDBCFEAFF01E3DB2A69
:10087000010EEF6EFD0EDBCFE9FFDB2AFE0EDBCFB4
:10088000EAFF01E3DB2AEF6AFD0EDBCFE9FFDB2A9B
:10089000FE0EDBCFEAFF01E3DB2A020EEF6EFD0E58
:1008A000DBCFE9FFDB2AFE0EDBCFEAFF01E3DB2A29
:1008B000EF6AFD0EDBCFE9FFDB2AFE0EDBCFEAFF9E
:1008C00001E3DB2AEF6AFD0EDBCFE9FFDB2AFE0E38
:1008D000DBCFEAFF01E3DB2AEF6AFD0EDBCFE9FFA6
:1008E000DB2AFE0EDBCFEAFF01E3DB2A080EEF6E08
:1008F000FD0EDBCFE9FFDB2AFE0EDBCFEAFF01E3D3
:10090000DB2AFB0EDBCFEFFFDBCF10F0FC0EDBCFE3
:1009100011F011C010F0116AFD0EDBCFE9FFDB2AE8
:10092000FE0EDBCFEAFF01E3DB2A10C0EFFFFF0E74
:10093000E76EF90EDBCF10F0FA0EDBCF11F0E750C7
:100940001016116AFD0EDBCFE9FFDB2AFE0EDBCFAE
:10095000EAFF01E3DB2A10C0EFFFF90EDBCF10F056
:10096000FA0EDBCF11F011C010F0116AFF0E101655
:10097000000E1116FD0EDBCFE9FFDB2AFE0EDBCFEA
:10098000EAFF01E3DB2A10C0EFFFFD0EDBCFE9FF3A
:10099000DB2AFE0EDBCFEAFF01E3DB2A010EEF6E5E
:1009A000FD0EDBCFE9FFDB2AFE0EDBCFEAFF01E322
:1009B000DB2AEF6AFD0EDBCFE9FFDB2AFE0EDBCF81
:1009C000EAFF01E3DB2AF80EDBCFEFFFDB28E66E60
:1009D000FD0EDBCFE9FFDB2AFE0EDBCFEAFF01E3F2
:1009E000DB2AE552E750EF6EFD0EDBCFE9FFDB2A95
:1009F000FE0EDBCFEAFF01E3DB2AEF6AFD0EDBCF61
:100A0000E9FFDB2AFE0EDBCFEAFF01E3DB2A010E62
:100A1000EF6EFD0EDBCF06F0FE0EDBCF07F002011E
:100A20001151065C106E12510758116E10C013F26E
:100A300011C2E9FF12C2EAFF13C2EFFF1351106E99
:100A4000116A10C0F3FF11C0F4FF00D0E552E7CFE8
:100A5000D9FF1200D9CFE6FFE1CFD9FFFD0EDBCFE2
:100A6000E9FFDB2AFE0EDBCFEAFF01E3DB2A090EFA
:100A7000EF6EFD0EDBCFE9FFDB2AFE0EDBCFEAFFD8
:100A800001E3DB2A040EEF6EFD0EDBCFE9FFDB2A6C
:100A9000FE0EDBCFEAFF01E3DB2AFC0EDBCFEFFF2C
:100AA000FD0EDBCFE9FFDB2AFE0EDBCFEAFF01E321
:100AB000DB2AEF6AFD0EDBCFE9FFDB2AFE0EDBCF80
:100AC000EAFF01E3DB2AFB0EDBCFEFFFFD0EDBCFFE
:100AD000E9FFDB2AFE0EDBCFEAFF01E3DB2AFA0E99
:100AE000DBCFEFFFFD0EDBCFE9FFDB2AFE0EDBCF16
:100AF000EAFF01E3DB2AF90EDBCFEFFFFD0EDBCFD0
:100B0000E9FFDB2AFE0EDBCFEAFF01E3DB2AF80E6A
:100B1000DBCFEFFFFD0EDBCFE9FFDB2AFE0EDBCFE5
:100B2000EAFF01E3DB2AEF6A090EF36EF46A00D0F4
:100B3000E552E7CFD9FF1200D9CFE6FFE1CFD9FFC9
:100B4000FD0EDBCFE9FFDB2AFE0EDBCFEAFF01E380
:100B5000DB2A060EEF6EFD0EDBCFE9FFDB2AFE0E71
:100B6000DBCFEAFF01E3DB2A240EEF6EFD0EDBCFC5
:100B7000E9FFDB2AFE0EDBCFEAFF01E3DB2A020EF0
:100B8000EF6EFD0EDBCFE9FFDB2AFE0EDBCFEAFFC7
:100B900001E3DB2AFB0EDBCFEFFFFD0EDBCFE9FF2E
:100BA000DB2AFE0EDBCFEAFF01E3DB2AFC0EDBCF04
:100BB000EFFFFD0EDBCFE9FFDB2AFE0EDBCFEAFF06
:100BC00001E3DB2AEF6A060EF36EF46A00D0E55209
:100BD000E7CFD9FF1200D9CFE6FFE1CFD9FFFD0E55
:100BE000DBCFE9FFDB2AFE0EDBCFEAFF01E3DB2AE6
:100BF000090EEF6EFD0EDBCFE9FFDB2AFE0EDBCF29
:100C0000EAFF01E3DB2A240EEF6EFD0EDBCFE9FFE6
:100C1000DB2AFE0EDBCFEAFF01E3DB2A030EEF6ED9
:100C2000FD0EDBCFE9FFDB2AFE0EDBCFEAFF01E39F
:100C3000DB2AFA0EDBCFEFFFFD0EDBCFE9FFDB2A6D
:100C4000FE0EDBCFEAFF01E3DB2AFC0EDBCFEFFF7A
:100C5000FD0EDBCFE9FFDB2AFE0EDBCFEAFF01E36F
:100C6000DB2A010EEF6EFD0EDBCFE9FFDB2AFE0E65
:100C7000DBCFEAFF01E3DB2AFB0EDBCFEFFFFD0E4C
:100C8000DBCFE9FFDB2AFE0EDBCFEAFF01E3DB2A45
:100C9000010EEF6EFD0EDBCFE9FFDB2AFE0EDBCF90
:100CA000EAFF01E3DB2AEF6A090EF36EF46A00D073
:100CB000E552E7CFD9FF1200D9CFE6FFE1CFD9FF48
:100CC000FD0EDBCFE9FFDB2AFE0EDBCFEAFF01E3FF
:100CD000DB2A090EEF6EFD0EDBCFE9FFDB2AFE0EED
:100CE000DBCFEAFF01E3DB2A050EEF6EFD0EDBCF63
:100CF000E9FFDB2AFE0EDBCFEAFF01E3DB2AFC0E75
:100D0000DBCFEFFFFD0EDBCFE9FFDB2AFE0EDBCFF3
:100D1000EAFF01E3DB2AFB0EDBCFEFFFFD0EDBCFAB
:100D2000E9FFDB2AFE0EDBCFEAFF01E3DB2AFA0E46
:100D3000DBCFEFFFFD0EDBCFE9FFDB2AFE0EDBCFC3
:100D4000EAFF01E3DB2AEF6AFD0EDBCFE9FFDB2AD6
:100D5000FE0EDBCFEAFF01E3DB2AF90EDBCFEFFF6C
:100D6000FD0EDBCFE9FFDB2AFE0EDBCFEAFF01E35E
:100D7000DB2AEF6AFD0EDBCFE9FFDB2AFE0EDBCFBD
:100D8000EAFF01E3DB2AEF6A090EF36EF46A00D092
:100D9000E552E7CFD9FF1200D9CFE6FFE1CFD9FF67
:100DA000FB0EDB50040F0201176FFD0EDBCFE9FFD6
:100DB000DB2AFE0EDBCFEAFF01E3DB2A17C2EFFFDF
:100DC000FD0EDBCFE9FFDB2AFE0EDBCFEAFF01E3FE
:100DD000DB2A250EEF6EFD0EDBCFE9FFDB2AFE0ED0
:100DE000DBCFEAFF01E3DB2A010EEF6EFD0EDBCF66
:100DF000E9FFDB2AFE0EDBCFEAFF01E3DB2AFB0E75
:100E0000DBCFEFFFFB0EDBCFF3FFDB06F350000978
:100E100013E0FC0EDBCFF3FFDB2AF350E66EFD0E92
:100E2000DBCFE9FFDB2AFE0EDBCFEAFF01E3DB2AA3
:100E3000E552E750EF6EE6D702011751106E116AC6
:100E400010C0F3FF11C0F4FF00D0E552E7CFD9FF87
:100E50001200D9CFE6FFE1CFD9FF020EE126020151
:100E6000116B126B136B146BFA0EDBCFE6FFFB0EEC
:100E7000DB50E552E724156FE66A030EE66E010EBD
:100E8000E66E020EE66EFC0EDBCFE6FFFD0EDB50DB
:100E900011250001106EFE0EDB500201122100012F
:100EA000116E10C0E6FF11C0E6FFD4DD126E070E12
:100EB000E15E1250F35002011127F450122311C2C7
:100EC00013F212C214F2FD0EDB5013250F01E96E6E
:100ED000FE0EDB50020114210F01EA6E070EEF6EC9
:100EE000010E0201116A1325106E14511122FD0E1C
:100EF000DB501024E96EFE0EDB501120EA6E240E4A
:100F0000EF6E020E116A1325106E14511122FD0EA0
:100F1000DB501024E96EFE0EDB501120EA6E010E4C
:100F2000EF6E030E116A1325106E14511122FD0E7F
:100F3000DB501024E96EFE0EDB501120EA6EEF6AE2
:100F4000040E116A1325106E14511122FD0EDB5090
:100F50001024E96EFE0EDB501120EA6E010EEF6EDA
:100F6000070E1127000E1223166B1551165D27E28E
:100F7000FB0EDB50165D02E3020E01D0010EDF6EA8
:100F8000DFCFE6FF1629E66EFD0EDB5011250001CE
:100F9000106EFE0EDB50020112210001116E10C016
:100FA000E6FF11C0E6FFC8DDE552E552E552E55225
:100FB000F35002011127F4501223162BD6D7166BCB
:100FC0001551165D2DE2FB0EDB50165D02E3010E9E
:100FD00001D0020EE76E010EE7CFDBFFDBCFE6FFAD
:100FE0001629E66E16291525E66EFD0EDB50112535
:100FF0000001106EFE0EDB50020112210001116E85
:1010000010C0E6FF11C0E6FFE6DD126E050EE15EE0
:101010001250F35002011127F4501223162BD0D78F
:10102000E66A200EE66E020EE66EF90EDBCFE6FFF4
:10103000FD0EDB5011250001106EFE0EDB5002018B
:1010400012210001116E10C0E6FF11C0E6FF34DE70
:10105000126E060EE15E1250F35002011127F45099
:101060001223FB0EDBCFE6FF010EE66EFD0EDB501A
:1010700011250001106EFE0EDB500201122100014D
:10108000116E10C0E6FF11C0E6FF86DEE552E552A4
:10109000E552E552F35002011127F4501223E66A9B
:1010A000200EE66E020EE66EF90EDB50810FE66E44
:1010B000FD0EDB5011250001106EFE0EDB5002010B
:1010C00012210001116E10C0E6FF11C0E6FFF4DD31
:1010D000126E060EE15E1250F35002011127F45019
:1010E0001223FA0EDBCFE6FFFB0EDB501525E66E72
:1010F000FD0EDB5011250001106EFE0EDB500201CB
:1011000012210001116E10C0E6FF11C0E6FF44DE9F
:10111000E552E552E552E552F35002011127F45031
:1011200012231351115D126E12511455136E050ED8
:10113000116A1325106E14511122FD0EDB5010247C
:10114000E96EFE0EDB501120EA6E12C0EFFF135164
:10115000115D126E12511455136E13C012F0136A02
:10116000060E116A1325106E14511122FD0EDB506C
:101170001024E96EFE0EDB501120EA6E12C0EFFF64
:1011800011C2F3FF12C2F4FF020EE15C03E200D0D1
:10119000E16AE552E16EE552E7CFD9FF1200D9CFFF
:1011A000E6FFE1CFD9FFFD0EDBCFE9FFDB2AFE0E24
:1011B000DBCFEAFF01E3DB2A090EEF6EFD0EDBCF8A
:1011C000E9FFDB2AFE0EDBCFEAFF01E3DB2A240E78
:1011D000EF6EFD0EDBCFE9FFDB2AFE0EDBCFEAFF71
:1011E00001E3DB2A010EEF6EFD0EDBCFE9FFDB2A08
:1011F000FE0EDBCFEAFF01E3DB2AEF6AFD0EDBCF59
:10120000E9FFDB2AFE0EDBCFEAFF01E3DB2A010E5A
:10121000EF6EFD0EDBCFE9FFDB2AFE0EDBCFEAFF30
:1012200001E3DB2A090EEF6EFD0EDBCFE9FFDB2ABF
:10123000FE0EDBCFEAFF01E3DB2AEF6AFD0EDBCF18
:10124000E9FFDB2AFE0EDBCFEAFF01E3DB2A010E1A
:10125000EF6EFD0EDBCFE9FFDB2AFE0EDBCFEAFFF0
:1012600001E3DB2AFC0EDBCFEFFF090EF36EF46A1D
:1012700000D0E552E7CFD9FF1200D9CFE6FFE1CF8A
:10128000D9FF020EE126090EDE6EDD6AE66A010E66
:10129000E66EE66EE66AFB0EDBCFE6FFFD0EDBCF09
:1012A00014F0FE0EDBCF15F0DE501424126EDD506C
:1012B0001520136E12C0E6FF13C0E6FF2AEC05F0FE
:1012C000166E070EE15E1650F3CF10F0F4CF11F05A
:1012D000D9CFE9FFDACFEAFF1050EE261150ED2208
:1012E000FB0EDB28E66EFD0EDBCF14F0FE0EDBCF2F
:1012F00015F0DE501424126EDD501520136E12C04E
:10130000E6FF13C0E6FF4BDFE552E552E552F3CFAF
:1013100010F0F4CF11F0D9CFE9FFDACFEAFF105087
:10132000EE261150ED22FA0EDBCFE6FFF80EDBCFF2
:10133000E6FFF90EDBCFE6FFFB0EDB28E66EFD0EC7
:10134000DBCF14F0FE0EDBCF15F0DE501424126E4E
:10135000DD501520136E12C0E6FF13C0E6FF79DDE5
:10136000166E060EE15E1650F3CF10F0F4CF11F0BA
:10137000D9CFE9FFDACFEAFF1050EE261150ED2267
:10138000FD0EDBCFE9FFDB2AFE0EDBCFEAFF01E338
:10139000DB2A090EEF6EFD0EDBCFE9FFDB2AFE0E26
:1013A000DBCFEAFF01E3DB2A020EEF6EDECF10F0A7
:1013B000DDCF11F0FF0E1016000E1116FD0EDBCF63
:1013C000E9FFDB2AFE0EDBCFEAFF01E3DB2A10C0D8
:1013D000EFFFDECF10F0DDCF11F011C010F0116A79
:1013E000FF0E1016000E1116FD0EDBCFE9FFDB2AF3
:1013F000FE0EDBCFEAFF01E3DB2A10C0EFFFFD0E9C
:10140000DBCFE9FFDB2AFE0EDBCFEAFF01E3DB2ABD
:10141000020EEF6EFD0EDBCFE9FFDB2AFE0EDBCF07
:10142000EAFF01E3DB2A010EEF6EFD0EDBCFE9FFE1
:10143000DB2AFE0EDBCFEAFF01E3DB2AFC0EDBCF6B
:10144000EFFFFD0EDBCFE9FFDB2AFE0EDBCFEAFF6D
:1014500001E3DB2AC00EEF6EFD0EDBCFE9FFDB2AD6
:10146000FE0EDBCFEAFF01E3DB2AFA0EEF6EDECFE2
:1014700010F0DDCF11F010C0F3FF11C0F4FF020E29
:10148000E15C03E200D0E16AE552E16EE552E7CFAC
:10149000D9FF1200D9CFE6FFE1CFD9FFFD0EDBCF98
:1014A00060F0FE0EDBCF61F0FB0EDBCF62F0FC0ED6
:1014B000DBCF63F0FA0EDBCF64F0F90EDBCF65F023
:1014C000F70EDBCF66F0F80EDBCF67F0F50EDBCF63
:1014D00068F0F60EDBCF69F06BEC11F0E552E7CF68
:1014E000D9FF120004014851600BE842E842E8428B
:1014F000E842E842000901E051D04951070A4DE0B5
:101500000B0A4BE0070A3CE0010A29E00B0A25E040
:10151000020A23E0030A1FE0080A11E0010A0DE0B5
:101520000F0A09E0030A01E038D00001010EAB6F99
:10153000040EB76F33D093D831D056D92FD00001D5
:10154000010EAB6FB90EAC6F000EAD6FB883B895DE
:10155000010EB06F23D06DD921D0B8D91FD00001B2
:10156000010EAB6F04014C510001AC6FAD6BBA0EB4
:10157000AC27000EAD23B883B895010EB06F0ED026
:101580000001010EAB6F04014C51EA6ABA0FE96E1B
:10159000000EEA224AC4EFFF01D000D01200D9CFDA
:1015A000E6FFE1CFD9FF020EE126FB0EDBCFDEFF27
:1015B000DBCFDDFFDF2A010E01E3DB2ADFCFE9FF0E
:1015C000DF2ADBCFEAFF01E3DB2A030EEF6EFD0E1D
:1015D000DBCFF6FFFE0EDBCFF7FF0800F55021E072
:1015E000FD0EDBCFF6FFDB2AFE0EDBCFF7FF01E3BC
:1015F000DB2A0800F550E66EDFCFE9FFDF2A010E97
:10160000DBCFEAFF01E3DB2AE552E750EF6EDFCFE5
:10161000E9FFDF2A010EDBCFEAFF01E3DB2AEF6AF5
:10162000D6D7DECF12F0DDCF13F0FB0EDB50125C0D
:10163000106EFC0EDB501358116EFB0EDBCFE9FF72
:10164000FC0EDBCFEAFF10C0EFFF020EE15C02E20E
:10165000E16AE552E16EE552E7CFD9FF1200D9CF3A
:10166000E6FFE1CFD9FF020EE126800E0401485DBE
:1016700001E0B0D04B51030A59E0010A33E0030AFC
:1016800001E0A8D00001010EAB6F600EAC6F260E1A
:10169000AD6F0201120E186F18510001B06FB16BDF
:1016A000B893B895010EE66E62C0E6FF63C0E6FF30
:1016B00060C0E6FF61C0E6FFE66A070EE66E1CEC5E
:1016C00004F0106E070EE15E1050F3CF18F2020125
:1016D00018510001B06FB16BAC6B070EAD6FB883E2
:1016E000B89578D00001010EAB6F65C0E6FF64C00D
:1016F000E6FF030EE66E010EE66E020EE66E200EAB
:10170000E66E070EE66EB9DD106E070EE15E105054
:10171000F3CF18F2020118510001B06FB16B200E27
:10172000AC6F070EAD6FB883B89554D00001010EB1
:10173000AB6F04014A5100081BE24A51020818E34A
:101740006A0EE66E000EE66E4A05E96EEA6AD89009
:10175000E936EA36660EE926000EEA22EECFE6FF0B
:10176000EFCFE6FF1CDFE552E552E552E55225D00A
:101770006A0EDE6E000EDD6E4A510AE10001040EB3
:101780006A6F030E6B6F090E6C6F040E6D6F15D0D0
:101790000001060E6A6F030E6B6F710E6C6F6D6B3E
:1017A0000A0E106E10C00CF04AC407F00AEC14F0D8
:1017B0000350300F00016E6F6F6B00016A0EAC6F4B
:1017C000000EAD6F6AC0B0F0B16BB0BFB169B88345
:1017D000B89500D0020EE15C02E2E16AE552E16EEA
:1017E000E552E7CFD9FF12000001010EAB6F0F0EDB
:1017F000E66E710EE66E0F0EE66E22DBE552E552E6
:10180000E552010EE66EBA0EE66E000EE66E18DBCD
:10181000E552E552E5524AC4B9F004014A5104E1E7
:101820000001050EB76F04D00001060EB76F1DDB77
:1018300012000401506B516B48511F0B020A16E055
:10184000030A10E0010A01E035D00001010EAB6F80
:1018500080A402D0040150810001B8A102D004018B
:10186000508328D00001010EAB6F24D00001010E7F
:10187000AB6F04014C510F0B080DF350116A000FB0
:10188000106E040E11224C51800B01E0010E040D6C
:10189000F35000011024AE6F000E1120AF6FAEC0E8
:1018A000E9FFAFC0EAFFEF50040B03E00401010EB3
:1018B000506F00D00001AB0508E1500EAC6F040E74
:1018C000AD6FB883B895020EB06F120004014A05DF
:1018D00010E148511F0B00090CE10001010EAB6F34
:1018E000030E0401495D03E10001B88102D000014B
:1018F000B89104014A513AE148511F0B020836E100
:101900004C510F0B000932E00001010EAB6F0401D6
:101910004C510F0B080DF350116A000F106E040E9E
:1019200011224C51800B01E0010E040DF350000117
:101930001024AE6F000E1120AF6F030E0401495D3D
:1019400007E1840EAEC0E9FFAFC0EAFFEF6E0ED034
:101950004CAF06D0AEC0E9FFAFC0EAFFEF6A06D0D9
:10196000880EAEC0E9FFAFC0EAFFEF6E12006C5008
:101970000CE16896040100513C0BE842E8420D0876
:1019800002E10ED801D021D808D0040E6C5C03E12E
:1019900068962BD802D0000E02D0010E00D01200A3
:1019A000D9CFE6FFE1CFD9FFE652040104BF046BB3
:1019B0000001B26BAA6BAB6BB06BB16B93DDEFD870
:1019C000E552E552E7CFD9FF1200020E0001AA5DF1
:1019D0000AE1A8D8040100BD03D0C80E006F02D0F0
:1019E000880E006F01D01ED91200040E0001B75DF1
:1019F0000AE14AC46EFF6E50000803E2050EB76F9D
:101A000002D0030EB76FAA0512E113D8020E00012F
:101A1000B25D04E10401840E046F08D0040104BD2A
:101A200003D0C80E046F02D0880E046F01D0FAD81C
:101A30001200D9CFE6FFE1CFD9FF020EE126000167
:101A4000080EB05D000EB1590EE2B0C0DEFFB1C0AD
:101A5000DDFFB25103E1010EB26F04D0B20502E125
:101A6000020EB26F03D0080EDE6EDD6A040104932D
:101A70000491010EDB500413DFCF05F4000EDB50A0
:101A80000001B05F010EDB50B15B500EAE6F040E73
:101A9000AF6FB851060BE842E8B2FC0900091DE13E
:101AA000D9CFE9FFDACFEAFFEE50ED1015E0ACC078
:101AB000F6FFADC0F7FF0800F550AEC0E9FFAFC0BC
:101AC000EAFFEF6EAE2B000EAF23AC2BAD23DF068B
:101AD000010E01E2DB06E4D71BD0D9CFE9FFDACF54
:101AE000EAFFEE50ED1014E0ACC0E9FFADC0EAFF34
:101AF000EF50AEC0E9FFAFC0EAFFEF6EAE2B000EB5
:101B0000AF23AC2BAD23DF06010E01E2DB06E5D7E8
:101B1000020EE15C02E2E16AE552E16EE552E7CFD6
:101B2000D9FF1200D9CFE6FFE1CFD9FF020EE1269F
:101B3000030E04010015E76E010EE7CFDBFF01C4C1
:101B4000DFFFDE500001B027DD50B123500EAC6F37
:101B5000040EAD6FD9CFE9FFDACFEAFFEE50ED10FA
:101B600014E0ACC0E9FFADC0EAFFEF50AEC0E9FF42
:101B7000AFC0EAFFEF6EAE2B000EAF23AC2BAD2350
:101B8000DF06010E01E2DB06E5D7020EE15C02E2B0
:101B9000E16AE552E16EE552E7CFD9FF12006D9898
:101BA0000001AB510BE10401080E016F480E026FFA
:101BB000040E036F840E006F046F33D0040148AF2E
:101BC00021D00001B05104014E5D0001B15104016A
:101BD0004F5904E24EC4B0F04FC4B1F02ADF000107
:101BE000010EAA6F0401080E016F480E026F040E69
:101BF000036F800E006F500E066F040E076FC80E45
:101C0000046F0FD00001020EAA6F0401056BC80E0D
:101C1000046F080E016F500E026F040E036FC80EA2
:101C2000006F1200D9CFE6FFE1CFD9FFE652020ED6
:101C30000001AA5D36E16D50100B33E00401015143
:101C4000106E116A080E101801E111502AE10051BE
:101C50003C0BE842E8420D0824E10051800B21E1F1
:101C6000480E026F040E036FDF6ADF50106E116AB8
:101C7000080E105C000E115813E2DF50EA6A500F94
:101C8000E96E040EEA22EF50E66EDF50EA6A480F72
:101C9000E96E040EEA22E552E750EF6EDF2AE5D73F
:101CA0000CD00001AA6B0401080E016F480E026FF0
:101CB000040E036F8C0E006F046BE552E552E7CF04
:101CC000D9FF120080A203D06DA60FD802D06DB646
:101CD00013D80001B70508E16DBA06D0686A696AD1
:101CE00069806988020EB76F12006D6A696A6D8635
:101CF0000001010EB76F12006D6A696A0001B76BCF
:101D000012007CEF0EF00001B75101E143D06850A2
:101D1000040B04E06950040B01E041D86DB23AD0E5
:101D20006850010B04E06950010B01E062D8685073
:101D3000100B04E06950100B01E02DD86850400BE7
:101D400004E06950400B01E042D86850200B04E0E9
:101D50006950200B01E03DD86850020B04E0695047
:101D6000020B01E044D8030E0001B75D01E212D07E
:101D7000B36B060EB35D0EE26850080B0AE06950C3
:101D8000080B07E0F4DD000901E168960001B32BC0
:101D9000F0D700D01200698468986D8212006D92AD
:101DA000699468A402D06894FCD712000001B8A11D
:101DB0000DD06D926D84080EB46F070EB56FB40729
:101DC000000EB55BB451B511FAE16D941200689C38
:101DD000120070A00AD0800E0401005D05E1840E9F
:101DE000045D02E18C0E006F7090689A12006A6ABE
:101DF00012006A6A686A9F0E6B6E7B0E696E6E6A6D
:101E00000F0EE66E710EE66E0F0EE66E19D8E552F5
:101E1000E552E552160E706E68A608D0689600006E
:101E200000000000000000000000F6D76D98FADE08
:101E30000001B8910001B96B0001030EB76F1200E9
:101E4000D9CFE6FFE1CFD9FFFD0EDBCFE9FFFE0ED4
:101E5000DBCFEAFFFC0EDB5004E0EE6AFC0EDB0693
:101E6000F9D7E552E7CFD9FF12000001B66B1E0E7D
:101E7000716E0401400E096F580E0A6F040E0B6F4D
:101E8000880E086F980E0E6F040E0F6F400E0C6FC9
:101E90001D0EE96E040EEA6E200EEF6E1E0EE96E48
:101EA000040EEA6ED80EEE6E040EED6E1C0EE96E98
:101EB000040EEA6E400EEF6E1A0E746E250EE96E79
:101EC000040EEA6E200EEF6E260EE96E040EEA6E28
:101ED000E00EEE6E040EED6E240EE96E040EEA6E58
:101EE000400EEF6E1200D9CFE6FFE1CFD9FFE652E8
:101EF000FC0EDB50400805E2400EF36EFC0EF3CF03
:101F0000DBFFDF6AFC0EDB50DF5C19E2DF50E76EBF
:101F1000FD0EDBCFE9FFFE0EDBCFEAFFE750E9263F
:101F2000000EEA22EF50E66EDF50EA6A980FE96E83
:101F3000040EEA22E552E750EF6EDF2AE3D7FC0EEB
:101F4000DBCF0DF4400E04010C170C7D880E0C1332
:101F5000E552E552E7CFD9FF1200D9CFE6FFE1CF36
:101F6000D9FF020EE126FE0EDB50040DF3CF12F076
:101F7000F4CF13F0000E1226040E1322FE0EDB50D7
:101F8000040D1250F324106E1350F420116E040E41
:101F90001026000E112210C0DEFF11C0DDFFDECFC3
:101FA000E9FFDDCFEAFFEE52FB0EDBCFEFFF0201D0
:101FB000116BFB0EDB50115D26E21151E76EFC0E3A
:101FC000DBCFE9FFFD0EDBCFEAFFE750E926000E8D
:101FD000EA22EF50E66E1151106E116ADECFE9FF72
:101FE000DDCFEAFF020EE926000EEA221050EE24B1
:101FF000E76E1150EE20EA6EE7CFE9FFE552E750B9
:10200000EF6E112BD6D7400E106EDECFE9FFDDCF7D
:10201000EAFF1050EF16DECFE9FFDDCFEAFFEF5009
:10202000400B400A01E0010E106EDECFE9FFDDCF6C
:10203000EAFF1050010BF36EF346F346F346F34606
:10204000F346F346BF0EEF14F310EF6E880E106EDA
:10205000DECFE9FFDDCFEAFF1050EF12020EE15CA8
:1020600002E2E16AE552E16EE552E7CFD9FF1200E4
:10207000D9CFE6FFE1CFD9FF020EE126FE0EDB50FD
:10208000040DF3CF12F0F4CF13F0000E1226040E5D
:102090001322FE0EDB50040D1250F324106E135069
:1020A000F420116E040E1026000E112210C0DEFF67
:1020B00011C0DDFFDECFE9FFDDCFEAFFEF50800B7F
:1020C00001E0010E106E020EE15C03E200D0E16A55
:1020D000E552E16E1050E552E7CFD9FF1200D9CF9B
:1020E000E6FFE1CFD9FF020EE126FE0EDB50040D24
:1020F000F3CF12F0F4CF13F0000E1226040E1322C9
:10210000FE0EDB50040D1250F324106E1350F42019
:10211000116E10C0DEFF11C0DDFF0201006BDECFCB
:10212000E9FFDDCFEAFFEE52EF50005D26E20051FD
:10213000106E116ADECFE9FFDDCFEAFF020EE9265D
:10214000000EEA221050EE24E76E1150EE20EA6EE7
:10215000E7CFE9FFEF50E66E0051E76EFC0EDBCFF4
:10216000E9FFFD0EDBCFEAFFE750E926000EEA2289
:10217000E552E750EF6E002BD2D7400E106EDECF47
:10218000E9FFDDCFEAFF1050EF16DECFE9FFDDCF2C
:10219000EAFFEF50400B400A01E0010E106EDECF67
:1021A000E9FFDDCFEAFF1050010BF36EF346F34673
:1021B000F346F346F346F346BF0EEF14F310EF6E0B
:1021C000880E106EDECFE9FFDDCFEAFF1050EF1270
:1021D000106E020EE15C02E2E16AE552E16E10501F
:1021E000E552E7CFD9FF1200D9CFE6FFE1CFD9FF03
:1021F000020EE126FE0EDB50040DF3CF12F0F4CFF9
:1022000013F0000E1226040E1322FE0EDB50040DF6
:102210001250F324106E1350F420116E10C0DEFF24
:1022200011C0DDFFDECFE9FFDDCFEAFFEF50800B0D
:1022300001E0010E106E020EE15C03E200D0E16AE3
:10224000E552E16E1050E552E7CFD9FF1200D9CF29
:10225000E6FFE1CFD9FF0001B66B040108BF30D023
:10226000FC0EDBCF10F00951D880105403E2FC0EB5
:1022700009C4DBFF0001B66BFC0EDB50B65D19E252
:10228000B651EA6A580FE96E040EEA22EF50E66E84
:10229000B651E76EFD0EDBCFE9FFFE0EDBCFEAFFA6
:1022A000E750E926000EEA22E552E750EF6EB62B22
:1022B000E3D70401400E096F0817087D880E081344
:1022C0000001B65100D0E552E7CFD9FF1200FADC89
:1022D0006FAE19DD120092829284140E6F6E0001AF
:0822E000B76BB86BB96B12007B
:0822E8000F0EC1121200D9CF44
:1022F000E6FFE1CFD9FF020EE1260201046B056B78
:102300000001BB6F010EBC6F020EC16FC26FC76FC1
:10231000060EC86F020ECD6F070ECE6FD36B040E84
:10232000D46FD96B050EDA6F010EDF6F040EE06F0C
:10233000010EE56F050EE66FD7DF9280010EC26ECB
:102340000E0EC112C190BC0EC06E9282380E931256
:10235000C60E9412F00E8C169516CE0EE66E270E53
:10236000E66EE40EE66E270EE66E050EE66EE66E8F
:102370001C0EE66E400EE66E320EE66E080EE66E3F
:102380004AEC0AF0106E0A0EE15E1050E00EF26E9A
:10239000880ED56E67EC11F014D9040EE66E38EC99
:1023A00010F0E552000901E0F5D780500201086FF6
:1023B000096B81500A6F0B6B82500C6F0D6B0E6BAB
:1023C0000F6B080E0FAF02D0D89003D00E5D000E39
:1023D0000F5901E3BBD00EC210F00FC211F0060E70
:1023E0001102F3CF11F01002F3CF10F0F4501126C8
:1023F000BB0E1026000E112210C0DEFF11C0DDFF43
:10240000DECFE9FFDDCFEAFFEF34EA6AFE0BEA3602
:10241000E96E080EE926020EEA22EECF12F0EFCFA7
:1024200013F0DECFE9FFDDCFEAFFEE52EF5012C02E
:1024300010F013C011F005E0D89011321032E8040A
:10244000FBE11050010B02E0000E01D0010E020171
:10245000106F105144E0DECFE9FFDDCFEAFF020E3E
:10246000E926000EEA22EF503AE10EC210F00FC248
:1024700011F0030E1102F3CF11F01002F3CF10F0A0
:10248000F4501126320E1026000E1122DECFE9FF85
:10249000DDCFEAFF020EE926000EEA2210C0EFFFB0
:1024A000090E006F900E016FDECFE9FFDDCFEAFF6E
:1024B000020EE926000EEA22EFCF02F2400E036F71
:1024C000040EE66E000EE66E020EE66E040EE66E7A
:1024D000ADEC0FF0E552E552E552E55266D0DECFA5
:1024E000E9FFDDCFEAFF020EE926000EEA22EF50F7
:1024F00029E0105127E1090E006F900E016FDECF29
:10250000E9FFDDCFEAFF020EE926000EEA22EFCF57
:1025100002F2036B040EE66E000EE66E020EE66E2D
:10252000040EE66EADEC0FF0E552E552E552E552D1
:10253000DECFE9FFDDCFEAFF020EE926000EEA2238
:10254000EF6A33D00E2B000E0F233BD763D8020166
:10255000046F8C920551045D066F076B800E0715A2
:1025600004E0066D071F000E0723073504E206513D
:102570000208000E075519E20B0E006FB00E016F36
:10258000030E026F04C203F2040EE66E000EE66E46
:10259000020EE66E040EE66EADEC0FF0E552E5526B
:1025A000E552E55204C205F28C82F4D6F3D6020E4F
:1025B000E15C02E2E16AE552E16EE552E7CFD9FF64
:1025C0001200080E0001F5150201116F126B82A2B4
:1025D0001281040E821403E1115101E0128182ACD8
:1025E0001283800E821403E1115101E0128380A84E
:1025F000128580AA1287100E811403E1115101E0A7
:102600001285200E811403E1115101E0128712C2DC
:102610008CFF1200C282C2B2FED7C450200DF3500C
:10262000600B106EC350E840E840E8401F0B1F0BE2
:1026300010100201116F115100D01200DACFE4FF27
:10264000E2CFDAFFE652480ED76EE40ED66E0001F6
:10265000F52B000EF623F294E552E5CFDAFF1100D8
:10266000120100020000000818082E0101000102FA
:10267000000109022000010103C032090400000228
:102680000103000407050102400020070581024004
:1026900000200403090440036F006D0069006E0010
:1026A0006F0020004D006900630072006F0063003E
:1026B0006800690070002000540065006300680035
:1026C0006E006F006C006F00670079002000490009
:1026D0006E0063002E0050036F006D0069006E00F5
:1026E0006F0020004D006900630072006F006300FE
:1026F000680069007000200055005300420020006F
:10270000440065006D006F00200042006F00610012
:1027100072006400200028004300290020003200DD
:102720003000300037007226722692269626D62672
:102730002A0EF66E080EF76E000EF86E0001090004
:10274000F550F06F0900F550F16F03E1F06701D02B
:102750003DD00900F550EB6F0900F550EC6F090012
:10276000F550ED6F09000900F550E96E0900F550CC
:10277000EA6E090009000900F550EE6F0900F550F6
:10278000EF6F09000900F6CFF2F0F7CFF3F0F8CFC2
:10279000F4F0EBC0F6FFECC0F7FFEDC0F8FF00016E
:1027A000EE5302E1EF5307E00900F550EE6EEE073D
:1027B000F8E2EF07F9D7F2C0F6FFF3C0F7FFF4C075
:0E27C000F8FF0001F007000EF15BBFD712001A
:0227CE006F6D2D
:1027D000696E6F203830333820636F6E74726F6C9F
:1027E0006C6572006F6D696E6F2E636F6D20707215
:0727F0006F64756374730050
:0827F80013EE00F023EE00F0E7
:10280000F86A0F9C98EC13F01FEC14F077EC11F0C1
:04281000FBD71200E0
:0C281400036A080EE76ED8900736033602
:102820000C50035C02E3036E072AE72EF7D7120071
:0E28300000EE00F00F0EEE6AEA62FDD7120015
:02283E00120086
:02284000000195
:020000040030CA
:0100000024DB
:010001000EF0
:010002003FBE
:010003001EDE
:010005008179
:010006008178
:010008000FE8
:01000900C036
:01000A000FE6
:01000B00E014
:01000C000FE4
:01000D0040B2
:00000001FF
